:020000040000FA
:2B000000FFFF62FF2500FFFFFFFFFFFFFFFFFFFFFFFFFFFFFFFFFFFFFFFFFFFFFFFFFFFFFFFFFFFFFFFFFFFFFFFFFF76
:2B002B006018866118DC6119966118866118067718860100000000188661188661188661188661188661188661808CAD
:2B00560040100441100AE1100E4110044110844210040100000000100441100441100441100441100441100441808C46
:2B008100000000000000000000000000000000000000000000000000000000000000000000000000000000000080E7ED
:2B00AC00000000000000000000000000000000000000000000000000000000000000000000000000000000000080E7C2
:2B00D700000000000000800008080000000000000000000000000000000000000000000000000000000000000080EFFF
:2B010200000000000000A00000000000000000000000000000000000000000000000000000000000000000000000CF63
:2B012D00000000000000000000000000000000000000000000000000000000000000000000000000000000000080E740
:2B015800000000000000000000000000000000000000000000000000000000000000000000000000000000000080E715
:2B018300000000000000000000000000000000000000000000000000000000000000000000000000000000000080E7EA
:2B01AE00000000000000000000000000000000000000000000000000000000000000000000000000000000000080E7BF
:2B01D900000000000000000000000000000000000000000000000000000000000000000000000000000000000080E794
:2B020400000000000000000000000000000000000000000000000000000000000000000000000000000000000080E768
:2B022F00000000000000000000000000000000000000000000000000000000000000000000000000000000000080E73D
:2B025A00000000000000000000000000000000000000000000000000000000000000000000000000000000000080E712
:2B028500000000000000000000000000000000000000000000000000000000000000000000000000000000000080E7E7
:2B02B000000000000000000000000000000000000000000000000000000000000000000000000000000000000080E7BC
:2B02DB00000000000000000000000000000000000000000000000000000000000000000000000000000000000080E791
:2B030600000000000000000000000000000000000000000000000000000000000000000000000000000000000080E765
:2B033100000000000000000000000000000000000000000000000000000000000000000000000000000000000080E73A
:2B035C00000000000000000000000000000000000000000000000000000000000000000000000000000000000080E70F
:2B038700000000000000000000000000000000000000000000000000000000000000000000000000000000000080E7E4
:2B03B200020000000000000000000000000000000000000000000000000000000000000000000000000000000008ED29
:2B03DD00000000000000000000000000000000000000000000000000000000000000000000000000000000000080E78E
:2B040800000000000000000000000000000000000000000000000000000000000000000000000000000000000080E762
:2B043300000000000000000000000000000000000000000000000000000000000000000000000000000000000080E737
:2B045E00000000000000000000000000000000000000000000000000000000000000000000000000000000000080E70C
:2B048900020000000000000000000000000000000000000000000000000000000000000000000000000000000008ED51
:2B04B400800008800008800008800008800008800008000000000020000220000220000220000220000220000280E7BA
:2B04DF00800008800008800008800008800008800008000000000020000220000220000220000220000220000280E78F
:2B050A00000000000000000000000000000000000000000000000000000000000000000000000000000000000080E75F
:2B053500020000000000000000000000000000000000000000000000000000000000000000000000000000000008EDA4
:2B056000000000000000000000000000000000000000000000000000000000000000000000000000000000000080E709
:2B058B00000000000000000000000000000000000000000000000000000000000000000000000000000000000080E7DE
:2B05B600000000000000000000000000000000000000000000000000000000000000000000000000000000000080E7B3
:2B05E100000000000000000000000000000000000000000000000000000000000000000000000000000000000080E788
:2B060C00020000000000000000000000000000000000000000000000000000000000000000000000000000000008EDCC
:2B063700000000000000000000000000000000000000000000000000000000000000000000000000000000000080E731
:2B066200000000000000000000000000000000000000000000000000000000000000000000000000000000000080E706
:2B068D00000000000000000000000000000000000000000000000000000000000000000000000000000000000080E7DB
:2B06B800020000000000000000000000000000000000000000000000000000000000000000000000000000000008ED20
:2B06E300000000000000000000000000000000000000000000000000000000000000000000000000000000000080E785
:2B070E00000000000000000000000000000000000000000000000000000000000000000000000000000000000080E759
:2B073900000000000000000000000000000000000000000000000000000000000000000000000000000000000080E72E
:2B076400000000000000000000000000000000000000000000000000000000000000000000000000000000000080E703
:2B078F00020000000000000000000000000000000000000000000000000000000000000000000000000000000008ED48
:2B07BA00000000000000000000000000000000000000000000000000000000000000000000000000000000000080E7AD
:2B07E500000000000000000000000000000000000000000000000000000000000000000000000000000000000080E782
:2B081000000000000000000000000000000000000000000000000000000000000000000000000000000000000080E756
:2B083B00020000000000000000000000000000000000000000000000000000000000000000000000000000000008ED9B
:2B086600000000000000000000000000000000000000000000000000000000000000000000000000000000000080E700
:2B089100000000000000000000000000000000000000000000000000000000000000000000000000000000000080E7D5
:2B08BC00000000000000000000000000000000000000000000000000000000000000000000000000000000000080E7AA
:2B08E700000000000000000000000000000000000000000000000000000000000000000000000000000000000080E77F
:2B091200020000000000000000000000000000000000000000000000000000000000000000000000000000000008EDC3
:2B093D00000000000000000000000000000000000000000000000000000000000000000000000000000000000080E728
:2B096800000000000000000000000000000000000000000000000000000000000000000000000000000000000080E7FD
:2B099300000000000000000000000000000000000000000000000000000000000000000000000000000000000080E7D2
:2B09BE00020000000000000000000000000000000000000000000000000000000000000000000000000000000008ED17
:2B09E900000000000000000000000000000000000000000000000000000000000000000000000000000000000080E77C
:2B0A1400000000000000000000000000000000000000000000000000000000000000000000000000000000000080E750
:2B0A3F00000000000000000000000000000000000000000000000000000000000000000000000000000000000080E725
:2B0A6A00000000000000000000000000000000000000000000000000000000000000000000000000000000000080E7FA
:2B0A9500020000000000000000000000000000000000000000000000000000000000000000000000000000000008ED3F
:2B0AC000000000000000000000000000000000000000000000000000000000000000000000000000000000000080E7A4
:2B0AEB00000000000000000000000000000000000000000000000000000000000000000000000000000000000080E779
:2B0B1600000000000000000000000000000000000000000000000000000000000000000000000000000000000080E74D
:2B0B4100020000000000000000000000000000000000000000000000000000000000000000000000000000000008ED92
:2B0B6C00000000000000000000000000000000000000000000000000000000000000000000000000000000000080E7F7
:2B0B9700000000000000000000000000000000000000000000000000000000000000000000000000000000000080E7CC
:2B0BC200000000000000000000000000000000000000000000000000000000000000000000000000000000000080E7A1
:2B0BED00000000000000000000000000000000000000000000000000000000000000000000000000000000000080E776
:2B0C1800020000000000000000000000000000000000000000000000000000000000000000000000000000000008EDBA
:2B0C4300000000000000000000000000000000000000000000000000000000000000000000000000000000000080E71F
:2B0C6E00000000000000000000000000000000000000000000000000000000000000000000000000000000000080E7F4
:2B0C9900000000000000000000000000000000000000000000000000000000000000000000000000000000000080E7C9
:2B0CC400020000000000000000000000000000000000000000000000000000000000000000000000000000000008ED0E
:2B0CEF00000000000000000000000000000000000000000000000000000000000000000000000000000000000080E773
:2B0D1A00000000000000000000000000000000000000000000000000000000000000000000000000000000000080E747
:2B0D4500000000000000000000000000000000000000000000000000000000000000000000000000000000000080E71C
:2B0D7000000000000000000000000000000000000000000000000000000000000000000000000000000000000080E7F1
:2B0D9B00020000000000000000000000000000000000000000000000000000000000000000000000000000000008ED36
:2B0DC600000000000000000000000000000000000000000000000000000000000000000000000000000000000080E79B
:2B0DF100000000000000000000000000000000000000000000000000000000000000000000000000000000000080E770
:2B0E1C00000000000000000000000000000000000000000000000000000000000000000000000000000000000080E744
:2B0E4700020000000000000000000000000000000000000000000000000000000000000000000000000000000008ED89
:2B0E7200000000000000000000000000000000000000000000000000000000000000000000000000000000000080E7EE
:2B0E9D00000000000000000000000000000000000000000000000000000000000000000000000000000000000080E7C3
:2B0EC800000000000000000000000000000000000000000000000000000000000000000000000000000000000080E798
:2B0EF300000000000000000000000000000000000000000000000000000000000000000000000000000000000080E76D
:2B0F1E00020000000000000000000000000000000000000000000000000000000000000000000000000000000008EDB1
:2B0F4900000000000000000000000000000000000000000000000000000000000000000000000000000000000080E716
:2B0F7400000000000000000000000000000000000000000000000000000000000000000000000000000000000080E7EB
:2B0F9F00000000000000000000000000000000000000000000000000000000000000000000000000000000000080E7C0
:2B0FCA00000000000000000000000000000000000000000000000000000000000000000000000000000000000080E795
:2B0FF500000000000000000000000000000000000000000000000000000000000000000000000000000000000080E76A
:2B102000800008800008800008800008800008800008000000000020000220000220000220000220000220000280E742
:2B104B00800008800008800008800008800008800008000000000020000220000220000220000220000220000280E717
:2B107600000000000000000000000000000000000000000000000000000000000000000000000000000000000080E7E8
:2B10A100000000000000000000000000000000000000000000000000000000000000000000000000000000000080E7BD
:2B10CC00000000000000000000000000000000000000000000000000000000000000000000000000000000000080E792
:2B10F700000000000000000000000000000000000000000000000000000000000000000000000000000000000080E767
:2B112200000000000000000000000000000000000000000000000000000000000000000000000000000000000080E73B
:2B114D00000000000000000000000000000000000000000000000000000000000000000000000000000000000080E710
:2B117800000000000000000000000000000000000000000000000000000000000000000000000000000000000080E7E5
:2B11A300000000000000000000000000000000000000000000000000000000000000000000000000000000000080E7BA
:2B11CE00000000000000000000000000000000000000000000000000000000000000000000000000000000000080E78F
:2B11F900000000000000000000000000000000000000000000000000000000000000000000000000000000000080E764
:2B122400000000000000000000000000000000000000000000000000000000000000000000000000000000000080E738
:2B124F00000000000000000000000000000000000000000000000000000000000000000000000000000000000080E70D
:2B127A00000000000000000000000000000000000000000000000000000000000000000000000000000000000080E7E2
:2B12A500000000000000000000000000000000000000000000000000000000000000000000000000000000000080E7B7
:2B12D000000000000000000000000000000000000000000000000000000000000000000000000000000000000080E78C
:2B12FB00000000000000000000000000000000000000000000000000000000000000000000000000000000000080E761
:2B132600000000000000000000000000000000000000000000000000000000000000000000000000000000000080E735
:2B135100000000000000000000000000000000000000000000000000000000000000000000000000000000000080E70A
:2B137C00000000000000000000000000000000000000000000000000000000000000000000000000000000000080E7DF
:2B13A700000000000000000000000000000000000000000000000000000000000000000000000000000000000080E7B4
:2B13D200000000000000000000000000000000000000000000000000000000000000000000000000000000000080E789
:2B13FD00000000000000000000000000000000000000000000000000000000000000000000000000000000000080E75E
:2B142800020000000000000000000000000000000000000000000000000000000000000000000000000000000080E532
:2B145300000000000000000000000000000000000000000000000000000000000000000000000000000000000080E707
:2B147E00000000000000000000000000000000000000000000000000000000000000000000000000000000000080E7DC
:2B14A900000000000000000000000000000000000000000000000000000000000000000000000000000000000080E7B1
:2B14D400000000000000000000000000000000000000000000000000000000000000000000000000000000000080E786
:2B14FF00080000000000000000000000000000000000000000000000000000000000000000000000000000000080EF4B
:2B152A00000000000000000000000000000000000000000000000000000000000000000000000000000000000080E72F
:2B155500000000000000000000000000000000000000000000000000000000000000000000000000000000000080E704
:2B158000000000000000000000000000000000000000000000000000000000000000000000000000000000000080E7D9
:2B15AB00000000000000000000000000000000000020000000000000000000000000000000000000000000000080C5B0
:2B15D600000000000000000000000000000000000030000000000000000000000000000000000000000000000080D466
:2B160100000000000000000000000000000000001002000000000000000000000000000000000000000000000080C666
:2B162C00020000000000000000000000000000000000000000000000000000000000000000000000000000000080E52C
:2B165700000000000000000000000000000000000000000000000000000000000000000000000000000000000008EF71
:2B168200000000000000000000000000000000000000000000000000000000000000000000000000000000000008EF46
:2B16AD00000000000000000000000000000000003002000000000000000000000000000000000000000000000008CC0C
:2B16D800000000000000000000000000000000000000000000000000000000000000000000000000000000000008EFF0
:2B170300020000000000000000000000000000000000000000000000000000000000000000000000000000000080E554
:2B172E00800008800008800008800008800008800008000000000020000220000220000220000220000220000280E72D
:2B175900800008800008800008800008800008800008000000000020000220000220000220000220000220000280E702
:2B178400000000000000000000000000000000000080000000000000000000000000000000000000000000000000E7D3
:2B17AF000200000000000000000000000000000000060000000000000000000000000000000000000000000000088D72
:2B17DA00020000000000000000000000000000000000000000000000000000000000000000000000000000000080E57D
:2B18050004000000000000000000000000000000001C010000000000000000000000000000000000000000000000BBDC
:2B183000020000000000000000000000000000000000020000000000000000000000000000000000000000000080E722
:2B185B00020000000000000000000000000000000018000000000000000000000000000000000000000000000000FC4C
:2B188600020000000000000000000000000000000018000000000000000000000000000000000000000000000088F4A1
:2B18B100000000000000000000000000000000000018000000000000000000000000000000000000000000000000FEF6
:2B18DC00000000000000000000000000000000000080000000000000000000000000000000000000000000000000E77A
:2B19070000000000000000000000000000000000003E000000000000000000000000000000000000000000000000BCBB
:2B193200020000000000000000000000000000000018000000000000000000000000000000000000000000000000FC74
:2B195D00000000000000000000000000000000000004100000000000000000000000000000000000000000000008BF84
:2B198800000000000000000000000000000000000018040000000000000000000000000000000000000000000088F29E
:2B19B300000000000000000000000000000000000020000000000000000000000000000000000000000000000008CD14
:2B19DE00000000000000000000000000000000000000000000000000000000000000000000000000000000000008EFE7
:2B1A0900020000000000000000000000000000000018000000000000000000000000000000000000000000000000FC9C
:2B1A3400000000000000000000000000000000000040000000000000000000000000000000000000000000000080A324
:2B1A5F00000000000000000000000000000000000006000000000000000000000000000000000000000000000080874F
:2B1A8A00000000000000000000000000000000000000100000000000000000000000000000000000000000000080F7AA
:2B1AB50002000000000000000000000000000000003C00000000000000000000000000000000000000000000008896AA
:2B1AE000020000000000000000000000000000000020000000000000000000000000000000000000000000000080C772
:2B1B0B00040000000000000000000000000000000018000000000000000000000000000000000000000000000000FA99
:2B1B3600020000000000000000000000000000000018000000000000000000000000000000000000000000000000FC6E
:2B1B6100020000000000000000000000000000000018000000000000000000000000000000000000000000000000FC43
:2B1B8C00020000000000000000000000000000000080000000000000000000000000000000000000000000000088ED37
:2B1BB70000000000000000000000000000000000001E0000000000000000000000000000000000000000000000009E47
:2B1BE200000000000000000000000000000000000018000000000000000000000000000000000000000000000000FEC2
:2B1C0D00000000000000000000000000000000000004010000000000000000000000000000000000000000000080A681
:2B1C3800020000000000000000000000000000000018020000000000000000000000000000000000000000000088F6E7
:2B1C6300000000000000000000000000000000000000000000000000000000000000000000000000000000000080E7EF
:2B1C8E00000000000000000000000000000000000000000000000000000000000000000000000000000000000080E7C4
:2B1CB900000000000000000000000000000000000018000000000000000000000000000000000000000000000000FEEA
:2B1CE400000000000000000000000000000000000000040000000000000000000000000000000000000000000080E36E
:2B1D0F000200000000000000000000000000000000060000000000000000000000000000000000000000000000088D0C
:2B1D3A00000000000000000000000000000000000000000000000000000000000000000000000000000000000080E717
:2B1D650000000000000000000000000000000000001C020000000000000000000000000000000000000000000000BC79
:2B1D9000000000000000000000000000000000000000010000000000000000000000000000000000000000000080E6C1
:2B1DBB00020000000000000000000000000000000018000000000000000000000000000000000000000000000088F467
:2B1DE600020000000000000000000000000000000018000000000000000000000000000000000000000000000000FCBC
:2B1E1100040000000000000000000000000000000018000000000000000000000000000000000000000000000000FA90
:2B1E3C00020000000000000000000000000000000000000000000000000000000000000000000000000000000080E514
:2B1E670002000000000000000000000000000000001E0200000000000000000000000000000000000000000000009E90
:2B1E9200020000000000000000000000000000000018040000000000000000000000000000000000000000000088F08F
:2B1EBD00000000000000000000000000000000000004000000000000000000000000000000000000000000000080A7CF
:2B1EE800000000000000000000000000000000000018010000000000000000000000000000000000000000000000FFB7
:2B1F1300000000000000000000000000000000000000000000000000000000000000000000000000000000000080E73C
:2B1F3E00020000000000000000000000000000000000000000000000000000000000000000000000000000000008ED81
:2B1F6900000000000000000000000000000000000018000000000000000000000000000000000000000000000000FE37
:2B1F9400000000000000000000000000000000000080000000000000000000000000000000000000000000000000E7BB
:2B1FBF00000000000000000000000000000000000026000000000000000000000000000000000000000000000080A5AC
:2B1FEA00000000000000000000000000000000000000000000000000000000000000000000000000000000000080E765
:2B20150002000000000000000000000000000000001C100000000000000000000000000000000000000000000088A446
:2B204000000000000000000000000000000000000000040000000000000000000000000000000000000000000080E30E
:2B206B00000000000000000000000000000000000038000000000000000000000000000000000000000000000000DC36
:2B209600000000000000000000000000000000000018000000000000000000000000000000000000000000000000FE09
:2B20C100020000000000000000000000000000000018000000000000000000000000000000000000000000000000FCDE
:2B20EC00020000000000000000000000000000000040000000000000000000000000000000000000000000000008A9D6
:2B21170004000000000000000000000000000000001E0000000000000000000000000000000000000000000000889261
:2B214200020000000000000000000000000000000018100000000000000000000000000000000000000000000088E4DC
:2B216D000200000000000000000000000000000000240000000000000000000000000000000000000000000000088F8A
:2B219800020000000000000000000000000000000038000000000000000000000000000000000000000000000000DE04
:2B21C300000000000000000000000000000000000000000000000000000000000000000000000000000000000080E78A
:2B21EE00000000000000000000000000000000000000000000000000000000000000000000000000000000000080E75F
:2B221900000000000000000000000000000000000018000000000000000000000000000000000000000000000050AB87
:2B224400000000000000000000000000000000000000000000000000000000000000000000000000000000000008EF78
:2B226F00000000000000000000000000000000000000000000000000000000000000000000000000000000000080E7DD
:2B229A00800008800008800008800008800008800008000000000020000220000220000220000220000220000280E7B6
:2B22C500800008800008800008800008800008800008000000000020000220000220000220000220000220000280E78B
:2B22F000000000000000000000000000000000003002000000000000000000000000000000000000000000000080C44D
:2B231B00000000000000000000000000000000000010000000000000000000000000000000000000000000000080F611
:2B234600000000000000000000000000000000000000000000000000000000000000000000000000000000000080E705
:2B237100000000000000000000000000000000000000000000000000000000000000000000000000000000000080E7DA
:2B239C00000000000000000000000000000000001012000000000000000000000000000000000000000000000080D79D
:2B23C700000000000000000000000000000000000004000000000000000000000000000000000000000000000080A7C0
:2B23F200000000000000000000000000000000000000090000000000000000000000000000000000000000000080EE49
:2B241D00000000000000000000000000000000000000000000000000000000000000000000000000000000000080E72D
:2B244800000000000000000000000000000000000080000000000000000000000000000000000000000000000000E702
:2B2473000A0000000000000000000000000000000000000000000000000000000000000000000000000000000080EDC7
:2B249E00000000000000000000000000000000000000000000000000000000000000000000000000000000000080E7AC
:2B24C900020000000000000000000000000000000000000000000000000000000000000000000000000000000080E581
:2B24F400000000000000000000000000000000000000000000000000000000000000000000000000000000000080E756
:2B251F00000000000000000000000000000000000010100000000000000000000000000000000000000000000080E60B
:2B254A00000000000000000000000000000000000000000000000000000000000000000000000000000000000080E7FF
:2B257500000000000000000000000000000000000000000000000000000000000000000000000000000000000080E7D4
:2B25A000000000000000000000000000000000000000000000000000000000000000000000000000000000000080E7A9
:2B25CB00000000000000000000000000000000000000000000000000000000000000000000000000000000000080E77E
:2B25F600080000000000000000000000000000000000000000000000000000000000000000000000000000000080EF43
:2B262100000000000000000000000000000000000000000000000000000000000000000000000000000000000080E727
:2B264C00100000000000000000000000000000000000000000000000000000000000000000000000000000000080F7DC
:2B267700000000000000008000000000000000000000000000000000000000000000000000000000000000000080EF49
:2B26A200000000000000000400000000000000000000000000000000000000000000000000000000000000000080A3E6
:2B26CD00000000000000000000000000000000000000000000000000000000000000000000000000000000000080E77B
:2B26F800000000000000000000000000000000000000000000000000000000000000000000000000000000000080E750
:2B272300000000000000000000000000000000000000000000000000000000000000000000000000000000000080E724
:2B274E00000000000000000000000000000000000000000000000000000000000000000000000000000000000080E7F9
:2B277900000000000000000000000000000000000000000000000000000000000000000000000000000000000080E7CE
:2B27A400100000000000000000000000000000000000000000000000000000000000000000000000000000000080F783
:2B27CF00000000000000000000000000000000000000000000000000000000000000000000000000000000000080E778
:2B27FA00000000000000000000000000000000000000000000000000000000000000000000000000000000000080E74D
:2B282500000000000000000000000000000000000000000000000000000000000000000000000000000000000080E721
:2B285000000000000000000000000000000000000000000000000000000000000000000000000000000000000080E7F6
:2B287B00000000000002000000080000000080000000000000000000000000000000000000000000000000000000CFD9
:2B28A600020000000002000000000000000000000000000000000000000000000000000000000000000000000008CD2E
:2B28D100020000000000000000000000000000000000000000000000000000000000000000000000000000000080E575
:2B28FC00040000000000000000000000000080000000000000000000000000000000000000000000000000000000E34A
:2B2927000200000000000000000C0000000000000000000000000000000000000000000000000000000000000080E90E
:2B295200020000000000000000000000000000000000000000000000000000000000000000000000000000000080E5F3
:2B297D00020000000000000000000000000000000000000000000000000000000000000000000000000000000008ED38
:2B29A800800008800008800008800008800008800008000000000020000220000220000220000220000220000280E7A1
:2B29D300800008800008800008800008800008800008000000000020000220000220000220000220000220000280E776
:2B29FE00000000000000000800000000000000000000000000000000000000000000000000000000000000000000E7BF
:2B2A2900020000000000600000000000000000000000000000000000000000000000000000000000000000000080851B
:2B2A5400000000000000000000000000000000000000000000000000000000000000000000000000000000000008EF60
:2B2A7F00000000000000C00301000000000000000000000000000000000000000000000000000000000000000088845C
:2B2AAA00000000000000004000000000000000000000000000000000000000000000000000000000000000000008EBCE
:2B2AD500000000000000800300000000000000000000000000000000000000000000000000000000000000000088D4F7
:2B2B0000020000000000800100000000000000000000000000000000000000000000000000000000000000000000FC2B
:2B2B2B00000000000000800100000000000000000000000000000000000000000000000000000000000000000000FE00
:2B2B5600000000000000000800000000000000000000000000000000000000000000000000000000000000000000E765
:2B2B8100000000000000E00300000000000000000000000000000000000000000000000000000000000000000000BC8A
:2B2BAC00020000000000801100000000000000000000000000000000000000000000000000000000000000000088F5EE
:2B2BD700000000000000400200000000000000000000000000000000000000000000000000000000000000000080858C
:2B2C0200000000000000800300000000000000000000000000000000000000000000000000000000000000000000DC48
:2B2C2D00000000000000000000000000000000000000000000000000000000000000000000000000000000000080E715
:2B2C5800000000000000000000000000000000000000000000000000000000000000000000000000000000000080E7EA
:2B2C8300020000000000800100000000000000000000000000000000000000000000000000000000000000000088F427
:2B2CAE00000000000000000000000000000000000000000000000000000000000000000000000000000000000080E794
:2B2CD90000000000000060080000000000000000000000000000000000000000000000000000000000000000000087E1
:2B2D0400000000000000004000000000000000000000000000000000000000000000000000000000000000000080E301
:2B2D2F00000000000000C00100000000000000000000000000000000000000000000000000000000000000000000BEFA
:2B2D5A00020000000000000001000000000000000000000000000000000000000000000000000000000000000008FD46
:2B2D8500020000000000800300000000000000000000000000000000000000000000000000000000000000000088D640
:2B2DB000020000000000800100000000000000000000000000000000000000000000000000000000000000000088F4F9
:2B2DDB00020000000000800100000000000000000000000000000000000000000000000000000000000000000088F4CE
:2B2E0600000000000000000000000000000000000000000000000000000000000000000000000000000000000080E73A
:2B2E31000000000000006080000000000000000000000000000000000000000000000000000000000000000000808F87
:2B2E5C00000000000000002000000000000000000000000000000000000000000000000000000000000000000080E5C6
:2B2E8700000000000000C003000000000000000000000000000000000000000000000000000000000000000000009CC1
:2B2EB200020000000000000000000000000000000000000000000000000000000000000000000000000000000008EDFE
:2B2EDD00020000000000802100000000000000000000000000000000000000000000000000000000000000000000FE29
:2B2F0800040000000000800100000000000000000000000000000000000000000000000000000000000000000000FA1F
:2B2F3300020000000000800100000000000000000000000000000000000000000000000000000000000000000000FCF4
:2B2F5E00020000000000000800000000000000000000000000000000000000000000000000000000000000000000E559
:2B2F8900020000000000E00100000000000000000000000000000000000000000000000000000000000000000088941E
:2B2FB400000000000000800100000000000000000000000000000000000000000000000000000000000000000000FE73
:2B2FDF00000000000000400201000000000000000000000000000000000000000000000000000000000000000080956F
:2B300A00000000000000804100000000000000000000000000000000000000000000000000000000000000000000FAE0
:2B303500020000000000000200000000000000000000000000000000000000000000000000000000000000000080C725
:2B306000020000000000000000000000000000000000000000000000000000000000000000000000000000000008ED4E
:2B308B00040000000000800100000000000000000000000000000000000000000000000000000000000000000088F21B
:2B30B600020000000000000000000000000000000000000000000000000000000000000000000000000000000008EDF8
:2B30E100020000000000E00900000000000000000000000000000000000000000000000000000000000000000008943D
:2B310C00020000000000804100000000000000000000000000000000000000000000000000000000000000000000F8DD
:2B313700000000000000400000000000000000000000000000000000000000000000000000000000000000000080A706
:2B316200000000000000800101000000000000000000000000000000000000000000000000000000000000000000EED2
:2B318D00000000000000000200000000000000000000000000000000000000000000000000000000000000000080C5D0
:2B31B800020000000000000000000000000000000000000000000000000000000000000000000000000000000008EDF5
:2B31E300000000000000800100000000000000000000000000000000000000000000000000000000000000000000FE42
:2B320E00000000000000000800000000000000000000000000000000000000000000000000000000000000000000E7A6
:2B323900000000000000600200000000000000000000000000000000000000000000000000000000000000000080A5E3
:2B326400000000000000001000000000000000000000000000000000000000000000000000000000000000000080E6C9
:2B328F00020000000000C003000000000000000000000000000000000000000000000000000000000000000000889631
:2B32BA00000000000000000200000000000000000000000000000000000000000000000000000000000000000080C5A2
:2B32E500000000000000800100000000000000000000000000000000000000000000000000000000000000000000FE3F
:2B331000000000000000800100000000000000000000000000000000000000000000000000000000000000000000FE13
:2B333B00000000000000800100000000000000000000000000000000000000000000000000000000000000000000FEE8
:2B336600020000000000000000000000000000000000000000000000000000000000000000000000000000000008ED45
:2B339100020000000000E081000000000000000000000000000000000000000000000000000000000000000000889C8A
:2B33BC00020000000000802100000000000000000000000000000000000000000000000000000000000000000088F6C5
:2B33E7000200000000004002000000000000000000000000000000000000000000000000000000000000000000088FE0
:2B341200000000000000800100000000000000000000000000000000000000000000000000000000000000000000FE10
:2B343D00000000000000002000000000000000000000000000000000000000000000000000000000000000000080E5DF
:2B346800000000000000000000000000000000000000000000000000000000000000000000000000000000000080E7D2
:2B3493000200000000008001000000000000000000000000000000000000000000000000000000000000000000A8D60D
:2B34BE00020000000000000000000000000000000000000000000000000000000000000000000000000000000028CFEA
:2B34E900000000000000000000000000000000000000000000000000000000000000000000000000000000000080E751
:2B351400800008800008800008800008800008800008000000000020000220000220000220000220000220000280E729
:2B353F00800008800008800008800008800008800008000000000020000220000220000220000220000220000280E7FE
:2B356A00000000000000008080060000000000000000000000000000000000000000000000000000000000000000E947
:2B359500000000000000000000040000000000000000000000000000000000000000000000000000000000000080E3A4
:2B35C000000000000000000000000000000000000000000000000000000000000000000000000000000000000080E779
:2B35EB00000000000000000000000000000000000020000000000000000000000000000000000000000000000080C550
:2B361600000000000000808080040000000000000020000000000000000000000000000000000000000000000080C1A4
:2B364100000000000000000200000000000000000000000000000000000000000000000000000000000000000080C517
:2B366C00000000000000800000000000000000000000000000000000000000000000000000000000000000000000EFC4
:2B369700000000000000000000000000000000000000000000000000000000000000000000000000000000000080E7A1
:2B36C200000000000000009000000000000000000000000000000000000000000000000000000000000000000080EEDF
:2B36ED00180000000000000000000000000000000000000000000000000000000000000000000000000000000080FF1B
:2B371800000000000000000000000000000000000000000000000000000000000000000000000000000000000080E71F
:2B374300100000000000000000000000000000000000000000000000000000000000000000000000000000000080F7D4
:2B376E00000000000000000000000000000000000000000000000000000000000000000000000000000000000080E7C9
:2B379900000000000000400000000000000000000000000000000000000000000000000000000000000000000080A79E
:2B37C400080000000000000000000000000000000000000000000000000000000000000000000000000000000080EF63
:2B37EF00000000000000002000000000000000000000000000000000000000000000000000000000000000000080E52A
:2B381A00000000000000000000000000000000000000000000000000000000000000000000000000000000000080E71C
:2B384500000000000000000000000000000000000000000000000000000000000000000000000000000000000080E7F1
:2B387000000000000000000800000000000000000000000000000000000000000000000000000000000000000000E73E
:2B389B00000000000000000000000000000000000000000000000000000000000000000000000000000000000080E79B
:2B38C600000000000000000000000000000000000000000000000000000000000000000000000000000000000080E770
:2B38F100000000000000000000000000000000000000000000000000000000000000000000000000000000000080E745
:2B391C00000000000000000000000000000000000000000000000000000000000000000000000000000000000080E719
:2B394700401004411004411004411004411004411004010000000010044110044110044110044110044110044180E7F2
:2B397200601886611886611886611886611886611886010000000018866118866118866118866118866118866180E7CF
:02399D00FFFF2A
:00000001FF
